:100000000C945D000C9485000C9485000C94850084
:100010000C9485000C9485000C9485000C9485004C
:100020000C9485000C9485000C9485000C9485003C
:100030000C9485000C9485000C9485000C9485002C
:100040000C9480170C9485000C94F0170C94CA172C
:100050000C9485000C9485000C9485000C9485000C
:100060000C9485000C94850000000008000201003B
:100070000003040700000000000000000000000072
:10008000250028002B0000000000240027002A0083
:10009000040404040404040402020202020203032E
:1000A0000303030301020408102040800102040836
:1000B0001020010204081020221811241FBECFEFC7
:1000C000D8E0DEBFCDBF12E0A0E0B1E0E4E0FEE3A7
:1000D00002C005900D92AA33B107D9F722E0AAE336
:1000E000B2E001C01D92A33FB207E1F710E0CDE5F9
:1000F000D0E004C02197FE010E94CD1DCC35D10770
:10010000C9F70E945B180C94001F0C940000EF923A
:10011000FF920F931F93CF93DF938B01EA01E88146
:10012000F981E284F384DB01ED91FC910680F78193
:10013000E02D61E070E0C8010995482F61E070E0B2
:10014000CE01F7010995E881F981E484F584D801AD
:10015000ED91FC910084F185E02D61E070E0C80133
:100160000995482F61E070E0CE01F7010995E8811B
:10017000F981E284F384D801ED91FC910680F78146
:10018000E02D62E070E0C8010995482F62E070E060
:10019000CE01F7010995E881F981E484F584D8015D
:1001A000ED91FC910084F185E02D62E070E0C801E2
:1001B0000995482F62E070E0CE01F7010995E881CA
:1001C000F981E688F788D801ED91FC910284F385E6
:1001D000E02D64E070E0C8010995482F64E070E00C
:1001E000CE01F7010995E881F981E688F788D80101
:1001F000ED91FC910284F385E02D6CE070E0C80184
:100200000995482F6CE070E0CE01F7010995E8816F
:10021000F981E688F788D801ED91FC910284F38595
:10022000E02D63E070E0C8010995482F61E070E0BF
:10023000CE01F7010995E881F981E688F788D801B0
:10024000ED91FC910284F385E02D61E070E0C8013E
:100250000995482F62E070E0CE01F7010995E88129
:10026000F981E688F788D801ED91FC910284F38545
:10027000E02D62E070E0C8010995482F63E070E06E
:10028000CE01F7010995E881F981E688F788D80160
:10029000ED91FC910284F385E02D60E070E0C801EF
:1002A0000995482F60E070E0CE01F7010995E881DB
:1002B000F981E688F788D801ED91FC910284F385F5
:1002C000E02D6DE070E0C8010995482F6DE070E009
:1002D000CE01F7010995E881F981E688F788D80110
:1002E000ED91FC910284F385E02D6EE070E0C80191
:1002F0000995482F6EE070E0CE01F7010995E8817D
:10030000F981E688F788D801ED91FC910284F385A4
:10031000E02D6BE070E0C8010995482F6BE070E0BC
:10032000CE01F7010995E881F981E688F788D801BF
:10033000ED91FC910284F385E02D6AE070E0C80144
:100340000995482F6AE070E0CE01F7010995E88130
:10035000F981E688F788D801ED91FC910284F38554
:10036000E02D68E070E0C8010995482F68E070E072
:10037000CE01F7010995E881F981E688F788D8016F
:10038000ED91FC910284F385E02D69E070E0C801F5
:100390000995482F69E070E0CE01F701DF91CF9118
:1003A0001F910F91FF90EF900994EF92FF920F939E
:1003B0001F93CF93DF938B01EA01E881F981E284F7
:1003C000F384DB01ED91FC910680F781E02D61E083
:1003D00070E0C8010995482F61E070E0CE01F70197
:1003E0000995E881F981E484F584D801ED91FC91C7
:1003F0000084F185E02D61E070E0C8010995482F87
:1004000061E070E0CE01F7010995E881F981E284AD
:10041000F384D801ED91FC910680F781E02D62E034
:1004200070E0C8010995482F62E070E0CE01F70145
:100430000995E881F981E484F584D801ED91FC9176
:100440000084F185E02D62E070E0C8010995482F35
:1004500062E070E0CE01F7010995E881F981E68854
:10046000F788D801ED91FC910284F385E02D64E0DA
:1004700070E0C8010995482F64E070E0CE01F701F3
:100480000995E881F981E688F788D801ED91FC911A
:100490000284F385E02D6CE070E0C8010995482FD7
:1004A0006CE070E0CE01F7010995E881F981E688FA
:1004B000F788D801ED91FC910284F385E02D60E08E
:1004C00070E0C8010995482F61E070E0CE01F701A6
:1004D0000995E881F981E688F788D801ED91FC91CA
:1004E0000284F385E02D63E070E0C8010995482F90
:1004F00062E070E0CE01F7010995E881F981E688B4
:10050000F788D801ED91FC910284F385E02D61E03C
:1005100070E0C8010995482F63E070E0CE01F70153
:100520000995E881F981E688F788D801ED91FC9179
:100530000284F385E02D62E070E0C8010995482F40
:1005400060E070E0CE01F7010995E881F981E68865
:10055000F788D801ED91FC910284F385E02D6DE0E0
:1005600070E0C8010995482F6DE070E0CE01F701F9
:100570000995E881F981E688F788D801ED91FC9129
:100580000284F385E02D6EE070E0C8010995482FE4
:100590006EE070E0CE01F7010995E881F981E68807
:1005A000F788D801ED91FC910284F385E02D6BE092
:1005B00070E0C8010995482F6BE070E0CE01F701AB
:1005C0000995E881F981E688F788D801ED91FC91D9
:1005D0000284F385E02D6AE070E0C8010995482F98
:1005E0006AE070E0CE01F7010995E881F981E688BB
:1005F000F788D801ED91FC910284F385E02D68E045
:1006000070E0C8010995482F68E070E0CE01F7015D
:100610000995E881F981E688F788D801ED91FC9188
:100620000284F385E02D69E070E0C8010995482F48
:1006300069E070E0CE01F701DF91CF911F910F913A
:10064000FF90EF900994EF92FF920F931F93CF9337
:10065000DF938B01EA01E881F981E284F384DB0115
:10066000ED91FC910680F781E02D61E070E0C8011A
:100670000995482F61E070E0CE01F7010995E88106
:10068000F981E484F584D801ED91FC910084F18531
:10069000E02D61E070E0C8010995482F61E070E04D
:1006A000CE01F7010995E881F981E284F384D8014C
:1006B000ED91FC910680F781E02D62E070E0C801C9
:1006C0000995482F62E070E0CE01F7010995E881B5
:1006D000F981E484F584D801ED91FC910084F185E1
:1006E000E02D62E070E0C8010995482F62E070E0FB
:1006F000CE01F7010995E881F981E688F788D801EC
:10070000ED91FC910284F385E02D64E070E0C80176
:100710000995482F64E070E0CE01F7010995E88162
:10072000F981E688F788D801ED91FC910284F38580
:10073000E02D6CE070E0C8010995482F6CE070E096
:10074000CE01F7010995E881F981E688F788D8019B
:10075000ED91FC910284F385E02D61E070E0C80129
:100760000995482F61E070E0CE01F7010995E88115
:10077000F981E688F788D801ED91FC910284F38530
:10078000E02D62E070E0C8010995482F62E070E05A
:10079000CE01F7010995E881F981E688F788D8014B
:1007A000ED91FC910284F385E02D63E070E0C801D7
:1007B0000995482F63E070E0CE01F7010995E881C3
:1007C000F981E688F788D801ED91FC910284F385E0
:1007D000E02D60E070E0C8010995482F60E070E00E
:1007E000CE01F7010995E881F981E688F788D801FB
:1007F000ED91FC910284F385E02D6DE070E0C8017D
:100800000995482F6DE070E0CE01F7010995E88168
:10081000F981E688F788D801ED91FC910284F3858F
:10082000E02D6EE070E0C8010995482F6EE070E0A1
:10083000CE01F7010995E881F981E688F788D801AA
:10084000ED91FC910284F385E02D6BE070E0C8012E
:100850000995482F6BE070E0CE01F7010995E8811A
:10086000F981E688F788D801ED91FC910284F3853F
:10087000E02D6AE070E0C8010995482F6AE070E059
:10088000CE01F7010995E881F981E688F788D8015A
:10089000ED91FC910284F385E02D68E070E0C801E1
:1008A0000995482F68E070E0CE01F7010995E881CD
:1008B000F981E688F788D801ED91FC910284F385EF
:1008C000E02D69E070E0C8010995482F69E070E00B
:1008D000CE01F701DF91CF911F910F91FF90EF9023
:1008E0000994EF92FF920F931F93CF93DF938B01A5
:1008F000EA01E881F981E284F384DB01ED91FC9166
:100900000680F781E02D60E070E0C8010995482F6E
:1009100060E070E0CE01F7010995E881F981E48497
:10092000F584D801ED91FC910084F185E02D60E023
:1009300070E0C8010995482F60E070E0CE01F70132
:10094000DF91CF911F910F91FF90EF9009944F92FB
:100950005F926F927F92AF92BF92CF92DF92EF92AF
:10096000FF920F931F93CF93DF93EB018A01DA017C
:10097000ED91FC91E284F384E881F9810680F781AE
:10098000E02D61E070E0CE010995482F61E070E054
:10099000C801F7010995D801ED91FC91E484F58433
:1009A000E881F9810084F185E02D61E070E0CE01FD
:1009B0000995482F61E070E0C801F7010995E881C9
:1009C000F9810680F781E02D62E070E0CE010995A3
:1009D000682F880F770B60587F4F072E000C880B0D
:1009E000990B0E94831C20E030E045E553E40E940F
:1009F000381D20E030E044E752E40E94D91B6B012F
:100A00007C01E881F9810084F185E02D62E070E0ED
:100A1000CE010995682F880F770B60587F4F072EFE
:100A2000000C880B990B0E94831C20E030E045E508
:100A300053E40E94381D20E030E044E752E40E9475
:100A4000D91B2B013C01D801ED91FC91A284B38408
:100A500020E030E04FE753E4C701B6010E94331DA8
:100A6000181664F020E030E040E053E4C701B6011E
:100A70000E94671B0E944B1C462F01C04FE762E09B
:100A800070E0C801F5010995D801ED91FC91E4846D
:100A9000F58420E030E04FE753E4C301B2010E9447
:100AA000331D181664F020E030E040E053E4C30149
:100AB000B2010E94671B0E944B1C462F01C04FE7EA
:100AC00062E070E0C801F7010995D801ED91FC9151
:100AD000E688F788E881F9810284F385E02D64E0F7
:100AE00070E0CE010995482F64E070E0C801F7017D
:100AF0000995D801ED91FC91E688F788E881F981A4
:100B00000284F385E02D6CE070E0CE010995482F5A
:100B10006CE070E0C801F7010995D801ED91FC91F6
:100B2000E688F788E881F9810284F385E02D61E0A9
:100B300070E0CE010995482F61E070E0C801F7012F
:100B40000995D801ED91FC91E688F788E881F98153
:100B50000284F385E02D62E070E0CE010995482F14
:100B600062E070E0C801F7010995D801ED91FC91B0
:100B7000E688F788E881F9810284F385E02D63E057
:100B800070E0CE010995482F63E070E0C801F701DD
:100B90000995D801ED91FC91E688F788E881F98103
:100BA0000284F385E02D60E070E0CE010995482FC6
:100BB00060E070E0C801F7010995D801ED91FC9162
:100BC000E688F788E881F9810084F185E02D62E00C
:100BD00070E0CE010995D82EE881F9810284F38571
:100BE000E02D6DE070E0CE01099541E0BDEBDB1634
:100BF0000CF440E0482B6DE070E0C801F701099566
:100C0000D801ED91FC91E688F788E881F9810680AA
:100C1000F781E02D62E070E0CE010995D82EE881E1
:100C2000F9810284F385E02D6EE070E0CE01099534
:100C300041E0BDEBDB160CF440E0482B6EE070E0C9
:100C4000C801F7010995D801ED91FC91E688F78874
:100C5000E881F9810284F385E02D6BE070E0CE013C
:100C60000995482F6BE070E0C801F7010995D8019C
:100C7000ED91FC91E688F788E881F9810284F3859B
:100C8000E02D6AE070E0CE010995482F6AE070E03F
:100C9000C801F7010995D801ED91FC91E688F78824
:100CA000E881F9810284F385E02D68E070E0CE01EF
:100CB0000995482F68E070E0C801F7010995D8014F
:100CC000ED91FC91E688F788E881F9810284F3854B
:100CD000E02D69E070E0CE010995482F69E070E0F1
:100CE000C801F701DF91CF911F910F91FF90EF9015
:100CF000DF90CF90BF90AF907F906F905F904F90BC
:100D000009940F931F93CF938C01C62F0E94511B00
:100D1000C81721F06C2FC8010E94591B8C2FCF914E
:100D20001F910F910895FC01918D228D892F90E0E4
:100D3000805C9F4F821B91098F739927089580E0F3
:100D400090E0892B29F00E94071781110C94000074
:100D50000895DC01ED91FC910284F385E02D6DE0B6
:100D600070E00994FC0197859F7121F490899F7729
:100D700081E009F080E00895FC0197859F719D3026
:100D800029F490899F7781E0903509F080E00895FB
:100D90009B0177FF02C0295F3F4F43E035952795C0
:100DA0004A95E1F7FC01E20FF31F278530E0CB0104
:100DB00068E070E00E94A51DA90102C05595479505
:100DC0008A95E2F7CA0181700895660F771F860F32
:100DD000971FFC01828980580895660F771F860F40
:100DE000971FFC01818980580895FC0113A608957E
:100DF000FC0183A50895860F971F4195FC0140874C
:100E00000895860F971FFC01408708959B01442396
:100E1000E9F077FF02C0295F3F4F53E035952795F2
:100E20005A95E1F7FC01E20FF31FCB0168E070E097
:100E30000E94A51D21E030E0A90102C0440F551F0A
:100E40008A95E2F7CA019281892B1DC077FF02C003
:100E5000295F3F4F43E0359527954A95E1F7FC011F
:100E6000E20FF31FCB0168E070E00E94A51D21E0B6
:100E700030E0A90102C0440F551F8A95E2F7CA016C
:100E800080959281892382830895660F771FFC01E4
:100E9000E60FF71F8FE7489F402D112440584583E8
:100EA00008956F5F7F4F660F771FFC01E60FF71FF6
:100EB0008FE7489F402D1124405842830895660FC4
:100EC000771F860F971F4058FC01458308956F5F79
:100ED0007F4F660F771F860F971F4058FC01428394
:100EE0000895FC01128280E883838483858386834E
:100EF0008783108611860895CF92DF92EF92FF923A
:100F00000F931F93CF93DF938C01EB017A01DC01E8
:100F100015968D919C9116978130910521F002973D
:100F200009F45DC014C0E881F9810088F189E02DE1
:100F3000CB010995882331F082E090E0F801968397
:100F40008583C3C1D80116961C921E921597D701AE
:100F5000ED91FC91C284D384E881F9810680F78108
:100F6000E02D60E070E0CE010995682F880F770BC7
:100F7000880B990B0E94831CAB01BC01C8010E9425
:100F80004611482F60E070E0C701F6010995D701CE
:100F9000ED91FC91C484D584E881F9810084F185C8
:100FA000E02D60E070E0CE010995682F880F770B87
:100FB000880B990B0E94831CAB01BC01C8010E94E5
:100FC0004611482F60E070E0C701F601DF91CF9134
:100FD0001F910F91FF90EF90DF90CF900994D8016F
:100FE0001396ED91FC9114973496EE0FFF1FE00FCE
:100FF000F11F4081518157FF02C04F5F5F4F5595F0
:101000004795D701ED91FC910284F385E02D60E0D6
:1010100070E0C7010995D8011396ED91FC911497E2
:101020003896EE0FFF1FE00FF11F4081518157FFEF
:1010300002C04F5F5F4F55954795D701ED91FC91E9
:101040000484F585E02D60E070E0C7010995E88132
:10105000F9810088F189E02DCE010995882309F4F2
:101060004DC1F8018781E881F9810284F385E02D83
:10107000882309F461C062E070E0CE010995811116
:1010800074C1E881F9810284F385E02D63E070E0AA
:10109000CE010995811169C1E881F9810284F38546
:1010A000E02D61E070E0CE01099581115EC1E8811B
:1010B000F9810284F385E02D60E070E0CE010995AE
:1010C000811153C1E881F9810284F385E02D68E044
:1010D00070E0CE010995811148C1E881F98102844F
:1010E000F385E02D69E070E0CE01099581113DC1E5
:1010F000E881F9810284F385E02D6AE070E0CE0199
:101100000995811132C1E881F9810284F385E02DCE
:101110006BE070E0CE010995811127C1E881F9816A
:101120000284F385E02D64E070E0CE010995811121
:101130001CC1F801178219C163E070E0CE01099566
:101140008823C1F0D8011396ED91FC911497EE0F0E
:10115000FF1FE00FF11F808591858230910514F00B
:10116000019702C081E090E09187808781E0F801DB
:101170008783FBC0E881F9810284F385E02D62E07A
:1011800070E0CE0109958823A1F0D8011396ED9166
:10119000FC911497EE0FFF1FE00FF11F20853185A2
:1011A00080899189019728173907F4F6C9010196BA
:1011B000DBCFE881F9810284F385E02D61E070E006
:1011C000CE0109958823A1F0D8011396ED91FC91E9
:1011D0001497EE0FFF1FE00FF11F208931898085E2
:1011E000918501968217930704F5C90101971DC0E7
:1011F000E881F9810284F385E02D60E070E0CE01A2
:1012000009958823A9F0D8011396ED91FC911497C4
:10121000EE0FFF1FE00FF11F808991898F3F91052D
:1012200014F4019602C08FEF90E0918B808B9ECFDB
:10123000E881F9810284F385E02D64E070E0CE015D
:101240000995882381F0D8011396ED91FC911497AC
:10125000EE0FFF1FE00FF11F118610868FE790E061
:10126000918B808B47C0E881F9810284F385E02D62
:101270006BE070E0CE010995882321F0F80114821B
:10128000138223C0E881F9810284F385E02D68E0B0
:1012900070E0CE010995882341F081E090E0D8010B
:1012A00014969C938E93139726C0E881F98102844B
:1012B000F385E02D6AE070E0CE010995882339F0CE
:1012C00082E090E0F8019483838381E051CFE8814C
:1012D000F9810284F385E02D69E070E0CE01099583
:1012E000882309F442C083E090E0D80114969C93CF
:1012F0008E93139781E017968C9337C08091DF020D
:101300009091E002892B61F17801B8E0EB0EF11CBD
:10131000C0E0D0E0F7016081F2E0EF0EF11C8091B7
:10132000DF029091E0028C0F9D1F0E948106809148
:10133000DF029091E0028C0F9D1FD70116966C91F1
:1013400001960E9481062296C830D10519F7809136
:10135000DF029091E002F801638108960E94810605
:10136000D80116961C921E921597DF91CF911F916E
:101370000F91FF90EF90DF90CF9008956F927F9242
:101380008F929F92AF92BF92CF92DF92EF92FF9295
:101390000F931F93CF93DF9300D000D0CDB7DEB76C
:1013A0008C01DC0191968C9191978111E5C088E0C8
:1013B000E2E1F1E01F9601900D928A95E1F7D801E4
:1013C000AE58BF4F80E090E067E070E041E050E051
:1013D0009C0127703327FB01E21BF30B3A0102C08B
:1013E000660C771CEA95E2F79301FC0133E0F59572
:1013F000E7953A95E1F7E00FF11F378523232D9309
:1014000001968034910521F7780162E2E60EF11C25
:1014100080E4D7011D928A95E9F71C8261E0CE0134
:1014200004960E9456106AE070E0C7010E94011104
:10143000C8018E549F4F2AE0FC0111922A95E9F7CA
:101440004701F70140E050E077E0C72ED12CA19191
:101450009A0163E0359527956A95E1F7200F311FD2
:10146000590162EBA60EB11C61E070E0A11102C04F
:1014700060E070E0DA01A770BB2736016A1A7B0AC8
:1014800001C0660F6A94EAF7D901AE54BF4F2C91A0
:10149000622BD5016C934F5F5F4F40355105B9F614
:1014A000F801EC54FF4F2081277F2083FC0130811D
:1014B000311108C0F801ED54FF4F3081311102C0E5
:1014C000222329F081E0D80191968C9306C04AE04E
:1014D00050E060E071E00E94F91E8AE0E0EFF1E088
:1014E000D801579601900D928A95E1F780E5F701B2
:1014F00011928A95E9F781E4898361E0CE01019632
:101500000E9456106AE070E0C7010E940111019725
:1015100079F58AE0F8017796DF011D928A95E9F75F
:1015200020E030E047E050E0F40161914F01F90123
:1015300093E0F595E7959A95E1F7E00FF11F81E0CB
:1015400090E0611102C080E090E0B90167707727F8
:101550003A01661A770A01C0880F6A94EAF79789F8
:10156000892B878B2F5F3F4F20353105E9F6B4C0BB
:10157000D80191961C92B0C07801B2E2EB0EF11C3A
:1015800080E4F70111928A95E9F780911A01909110
:101590001B01A0911C0189839A83AB8363E0CE0178
:1015A00001960E94561068E070E0C7010E94011188
:1015B000D8019A968C91882309F48CC020E4F70115
:1015C000C8018E589F4FDC0101900D922A95E1F7DA
:1015D00028E0F8013F96DF011D922A95E9F7DC012A
:1015E00020E030E047E050E06D91F90183E0F595AF
:1015F000E7958A95E1F7E00FF11F81E090E0611136
:1016000002C080E090E0B901677077273A01661A5E
:10161000770A01C0880F6A94EAF79785892B878734
:101620002F5F3F4F20343105F9F662EF71E0F8018A
:1016300020E030E0DB015D91BD01818990E0418DCA
:10164000450F841B910947FD939597FD07C08F3F78
:10165000910529F024F08FEF90E001C080E0818BAC
:10166000A8014E575F4F982F9078DA019C934F5FF7
:101670005F4F982F9074DA019C934F5F5F4F982FC4
:101680009072DA019C934F5F5F4F982F9071DA014F
:101690009C934F5F5F4F982F9870DA019C934F5F38
:1016A0005F4F982F9470DA019C934F5F5F4F982F94
:1016B0009270DA019C934F5F5F4F8170DA018C93D7
:1016C0002F5F3F4F3196085F1F4F2630310509F0DD
:1016D000B1CF02C0F80111A20F900F900F900F90A0
:1016E000DF91CF911F910F91FF90EF90DF90CF90FE
:1016F000BF90AF909F908F907F906F9008950C94C3
:101700006B1E0F931F93CF93DF93CDB7DEB7289750
:101710000FB6F894DEBF0FBECDBF8C01FC01E95BB4
:10172000FE4F8081833440F4813408F045C0882323
:1017300031F08034C9F053C08F3F09F050C089E2C6
:10174000F8018283138280E2848340E063E0C80171
:1017500002960E94250F81E0F80183A760E070E007
:10176000C8010E94DA0F3BC080913A0281110DC07E
:1017700028E0C8010296FC01D801939601900D92D1
:101780002A95E1F741E068E00DC088E0F801B396E2
:10179000DE01119601900D928A95E1F741E068E033
:1017A000CE0101960E94250F61E070E0C8010E9401
:1017B000DA0F80933A0213C0F801128280E8838323
:1017C00084838583868387831086118681E0828760
:1017D000838741E06AE0C80102960E94250F28969F
:1017E0000FB6F894DEBF0FBECDBFDF91CF911F9132
:1017F0000F91089560E070E00C94DA0FFC01848D85
:10180000DF01A80FB11DA35ABF4F2C91848D90E02A
:1018100001968F739927848FA689B7892C93A08905
:10182000B1898C91837080648C93938D848D98138F
:1018300006C00288F389E02D80818F7D8083089522
:10184000CF92DF92EF92FF920F931F93CF93DF938C
:10185000EC011A8281E291E0998388831C821B82C9
:10186000198618868FE790E0998B888B1B861A86DD
:101870009B8B8A8B1D861C869D8B8C8B1F861E8660
:101880009F8B8E8B0091DF021091E00201151105F4
:1018900009F05DC082E00E94640D8C019093E0022B
:1018A0008093DF02009779F569E070E082E00E94A2
:1018B000D90C9093E0028093DF02892B09F46BC06E
:1018C00000E010E08091DF029091E00260E0800F84
:1018D000911F0E9481068091DF029091E002800FAB
:1018E000911F6FE701960E9481060E5F1F4F08301F
:1018F000110541F78091DF029091E00260E00896C7
:101900000E94810648C008960E94511B90E09C836B
:101910008B837E0188E0E80EF11C6E01E0E1CE0EC3
:10192000D11CC8010E94511B90E0F7018193919353
:101930007F01C80101960E94511B90E0F701978337
:1019400086830E5F1F4FCE14DF0459F724C0C801F1
:1019500008960E94511B90E09C838B837E01F8E0E7
:10196000EF0EF11C6E0180E1C80ED11CC8010E946F
:10197000511B90E0F701819391937F01C80101967B
:101980000E94511B90E0F701978386830E5F1F4FE3
:10199000EC14FD0459F781E090E09E838D83DF9184
:1019A000CF911F910F91FF90EF90DF90CF9008950E
:1019B00008958F929F92AF92BF92CF92DF92EF9253
:1019C000FF920F931F93CF93DF93C82E5B01E0909C
:1019D0004002F0904102C0E0D0E00AE010E0EC16D6
:1019E000FD060CF462C0C8010E94511B98012E5FD5
:1019F0003F4F49018F3F21F0EC16FD0609F04CC026
:101A0000C4010E94511BD82EEC16FD0651F090E047
:101A10008A159B050CF440C09C2F8D2FE701E92E01
:101A2000F82E6C2DC8010E94810660E0C801019665
:101A30000E9481060D5F1F4FEC16FD06A1F08D2D53
:101A400090E00297A816B9068CF47801EA0CFB1C0A
:101A50006FEFC7010E9481066D2D6A196350C7019F
:101A600002960E94810621966A2D01C06D2DC40147
:101A70000E94810680914002909141028C179D073F
:101A800049F0D0934102C09340026C2F81E090E076
:101A90000E948106C8010BC0C4010E94511B90E046
:101AA0000396080F191F21969ACF80E090E0DF91EE
:101AB000CF911F910F91FF90EF90DF90CF90BF904B
:101AC000AF909F908F900895DF92EF92FF920F93C7
:101AD0001F93CF93DF93D82EE0904002F090410205
:101AE00000E010E0CAE0D0E00E151F05CCF4CE01F6
:101AF0000E94511BD81209C0CE0101960E94511BB1
:101B0000811103C0CE0103960DC0CE0102960E9442
:101B1000511B90E00396C80FD91F0F5F1F4FE4CFF2
:101B200080E090E0DF91CF911F910F91FF90EF90B7
:101B3000DF9008950F931F93CF93DF93EC018B01F8
:101B40008E819F81009721F00E946B1E1F821E8252
:101B50008A819B81009711F00E946B1E1B830A8370
:101B6000DF91CF911F910F9108952F923F924F9245
:101B70005F926F927F928F929F92AF92BF92CF921D
:101B8000DF92EF92FF920F931F93CF93DF93CDB726
:101B9000DEB728970FB6F894DEBF0FBECDBF9E8389
:101BA0008D836A017B0120E030E040E053E4C7010F
:101BB000B6010E94331D181654F420E030E040E8CE
:101BC00053E4C701B6010E94671B6B017C0120E052
:101BD00030E0A901C701B6010E94D41B87FF0BC0EA
:101BE000F7FAF094F7F8F094812C912C90E8A92E54
:101BF0009FEBB92E13C020E030E0A901C701B60168
:101C00000E94D41B882339F0812C912C80E8A82EC7
:101C10008FE3B82E03C0812C912C5401ED81FE81FD
:101C200027803084B101032C000C880B990B0E9493
:101C3000831C2B013C01A70196010E94D41BED815E
:101C4000FE8118160CF4B5C001851285B801012E6D
:101C5000000C880B990B0E94831C69837A838B8309
:101C60009C83A70196010E94331D18160CF041C0F9
:101C7000ED81FE810584F685E02DFA83E983ED810F
:101C8000FE816385748529813A81621B730B072E5F
:101C9000000C880B990B0E94831C6D837E838F83BD
:101CA0009887A3019201C701B6010E94671B9B019F
:101CB000AC016D817E818F8198850E94381D6B01FA
:101CC0007C01B80162197309072E000C880B990B6F
:101CD0000E94831C9B01AC01C701B6010E94D91B65
:101CE0006B017C01E981FA81BF01FF0F880B990B21
:101CF00040C020E030E04EEF52E4C701B6010E9440
:101D0000D41B87FF3DC0ED81FE81238434846FE7BF
:101D100070E062197309072E000C880B990B0E9462
:101D2000831C2B013C0129813A814B815C81C701D5
:101D3000B6010E94671B9B01AC01C301B2010E9466
:101D4000381D6B017C012FE730E0201B310BB901FE
:101D5000330F880B990B0E94831C9B01AC01C701B8
:101D6000B6010E94D91B6B017C01B101330C880BB9
:101D7000990B0E94831C9B01AC01C701B60116C0E0
:101D800020E030E04EEF52E4C701B6010E94671B2D
:101D900020E030E0A9010E94381D20E030E0A901D8
:101DA0000E94D91B20E030E04EEF52E40E94681BF5
:101DB00010C065857685072E000C880B990B0E9454
:101DC000831CA70196010E94381DA30192010E9465
:101DD000D91BA50194010E94381D6B017C0120E0F4
:101DE00030E040E053EC0E94D41B87FD10C020E09F
:101DF00030E04EEF52E4C701B6010E94331D1816C1
:101E00004CF0C701B6010E944B1CCB0105C080E815
:101E10009FEF02C08FE790E028960FB6F894DEBFE0
:101E20000FBECDBFDF91CF911F910F91FF90EF902B
:101E3000DF90CF90BF90AF909F908F907F906F90EA
:101E40005F904F903F902F900895FC0128E0539AA7
:101E5000808190E0880F892F881F990B892B09F4C6
:101E600030C0000000000000000000000000000082
:101E70000000539800000000000000000000000077
:101E80000000000000000000000000000000000052
:101E90000000000000000000000000000000000042
:101EA0000000000000000000000000000000000032
:101EB0000000000000000000000000000000000022
:101EC00030C0000000000000000000000000000022
:101ED0000000000000000000000000000000000002
:101EE00000000000000000000000000000000000F2
:101EF00000000000000000000000000000000000E2
:101F000000000000000000000000000000000000D1
:101F100000000000000000000000000000000000C1
:101F20005398215069F000000000000000000000FC
:101F300000000000000000008081880F808387CFB0
:101F40000000000000000000615031F000000000BF
:101F50000000000031967ACF000000000000000071
:101F60000000000000000000539A00000000000084
:101F70000000000000000000000000000000000061
:101F80000000000000000000442391F00000000069
:101F90000000000000000000000000000000000041
:101FA0000000000000000000000000000000000031
:101FB00053980895CF93DF93DC01EC01CB5BDE4FA8
:101FC000FC01E95BFE4F808190E099838883108259
:101FD0001616170694F484EC99E04B9906C081E03C
:101FE0009B968C9388E090E01AC00197B1F79B967E
:101FF0008C919B97882309F454C09B968C918111F6
:102000000AC080E290E04B9902C080E290E0019724
:1020100018161906C4F388E090E04B99FECF000033
:1020200000000000000000000000000000000000B0
:1020300000000000000000000000000000000000A0
:102040000000000000000000000000000000000090
:102050000000000000000000000000000000000080
:10206000000000000000000000004B9B03C0208126
:1020700021602083019731F02081220F20834B9B28
:10208000FECFCBCF4B9BFECF8CE090E04B9902C0B4
:102090008CE090E0019718161906C4F381E090E0F7
:1020A00002C080E090E0DF91CF910895FC0128E02C
:1020B0008AB180638AB9808190E0880F892F881F58
:1020C000990B892B09F432C00000000000000000C9
:1020D00000000000000000008AB18F7C8AB9000077
:1020E00000000000000000000000000000000000F0
:1020F00000000000000000000000000000000000E0
:1021000000000000000000000000000000000000CF
:1021100000000000000000000000000000000000BF
:102120000000000000000000000032C000000000BD
:10213000000000000000000000000000000000009F
:10214000000000000000000000000000000000008F
:10215000000000000000000000000000000000007F
:10216000000000000000000000000000000000006F
:10217000000000000000000000000000000000005F
:10218000000000000000000000008AB18F7C8AB9C6
:10219000215069F000000000000000000000000075
:1021A0000000000000008081880F808381CF000044
:1021B000000000000000615031F00000000000004D
:1021C0000000319674CF0000000000000000000005
:1021D0000000000000008AB180638AB9000000009E
:1021E00000000000000000000000000000000000EF
:1021F000000000000000000000008AB18F7C8AB956
:102200000895FC01660F660F660F9FE329B12073E6
:1022100029F09150D9F780E090E008950000000087
:1022200000000000000000000000000000000000AE
:10223000000000000000000000000000000000009E
:10224000000000000000000000000000000000008E
:10225000000000000000000000000000000000007E
:10226000000000000000000099B19073919361504C
:1022700051F09FE329B1207309F0C7CF9150D1F7F6
:1022800082E090E0089581E090E008954F925F929F
:102290006F927F928F929F92AF92BF92CF92DF9276
:1022A000EF92FF92CF93DF93EC016A017B0120E074
:1022B00030E040E053E4C701B6010E94331D181618
:1022C00054F420E030E040E853E4C701B6010E9436
:1022D000671B6B017C0120E030E0A901C701B6015A
:1022E0000E94D41B87FF0BC0F7FAF094F7F8F09424
:1022F000812C912C40E8A42E4FEBB42E13C020E08B
:1023000030E0A901C701B6010E94D41B882339F02F
:10231000812C912C30E8A32E3FE3B32E03C0812CF7
:10232000912C54018B819C81880F991FC80FD91F54
:1023300068857985072E000C880B990B0E94831CF9
:102340002B013C01A70196010E94331D87FF44C069
:10235000A3019201C701B6010E94671B6B017C01BA
:10236000A301920160E070E08EEF92E40E94671B8F
:102370009B01AC01C701B6010E94D91B6B017C0116
:1023800068897989072E000C880B990B0E94831CA1
:102390009B01AC01C701B6010E94381DA501940143
:1023A0000E94381D6B017C0120E030E040E053ECDE
:1023B0000E94D41B87FD13C020E030E04EEF52E4B2
:1023C000C701B6010E94331D181664F0C701B6019B
:1023D0000E944B1CCB0108C080E090E005C080E863
:1023E0009FEF02C08FE790E0DF91CF91FF90EF90D9
:1023F000DF90CF90BF90AF909F908F907F906F9025
:102400005F904F900895CF93DF9390E0FC01EC55DF
:10241000FF4F2491FC01E057FF4F84918823C1F0C6
:1024200090E0880F991FFC01EA57FF4FC591D491A6
:10243000FC01E458FF4FA591B4919FB7F8948881AF
:10244000E22FE0958E2388838C91E823EC939FBF45
:10245000DF91CF91089590E0FC01E859FF4F24915E
:10246000FC01EC55FF4F3491FC01E057FF4FE49124
:10247000EE23B9F1222339F1233091F038F42130E1
:10248000A9F0223001F584B58F7D12C0273091F07C
:102490002830A1F02430B9F4809180008F7D03C0F2
:1024A000809180008F77809380000DC084B58F77F6
:1024B00084BD09C08091B0008F7703C08091B000C7
:1024C0008F7D8093B000F0E0EE0FFF1FE458FF4FC8
:1024D000A591B4919FB7F8948C91309538233C9393
:1024E0009FBF0895682F82E492E00C9411173FB7C4
:1024F000F89480913B0290913C02A0913D02B091F2
:102500003E0226B5A89B05C02F3F19F00196A11DDC
:10251000B11D3FBFBA2FA92F982F8827820F911D79
:10252000A11DB11DBC01CD0142E0660F771F881FC0
:10253000991F4A95D1F708952091E3023091E40262
:102540002115310529F0682FC90101960C948106E7
:102550000895682F8091E3029091E402009711F0B2
:102560000C9481060895DF92EF92FF920F931F93D0
:10257000CF93DF93EC018B017A018C819D818130B7
:10258000910521F0029709F471C011C0DB01ED91B2
:10259000FC910088F189E02DCB010995882329F071
:1025A00082E090E09D838C83DDC11D821C82D80176
:1025B000ED91FC910680F781E02D60E070E0C801AC
:1025C0000995D801ED91FC910084F185E02D60E042
:1025D00070E0C8010995D801ED91FC910680F78162
:1025E000E02D60E070E0C8010995682F880F770B37
:1025F000880B990B0E94831CAB01BC01CE010E9489
:10260000B50DD82ED801ED91FC910084F185E02D17
:1026100060E070E0C8010995682F880F770B880B80
:10262000990B0E94831CAB01BC01CE010E94B50D29
:10263000C82FD701ED91FC910284F385E02D4D2D3B
:1026400060E070E0C7010995D701ED91FC91048429
:10265000F585E02D4C2F60E070E0C701DF91CF9150
:102660001F910F91FF90EF90DF900994AF81B88593
:10267000A55CBE4FFA0180819181FC0122853385E2
:102680004C9160E070E0C701F9010995A985BA8510
:10269000A55CBE4FF70180819181FC0124853585C1
:1026A0004C9160E070E0C701F9010995D801ED9106
:1026B000FC910088F189E02DC8010995882309F46F
:1026C00054C18E81D801ED91FC910284F385E02DF7
:1026D000882309F468C062E070E0C801099581119F
:1026E0005FC1D801ED91FC910284F385E02D63E098
:1026F00070E0C8010995811153C1D801ED91FC9199
:102700000284F385E02D61E070E0C8010995811134
:1027100047C1D801ED91FC910284F385E02D60E082
:1027200070E0C801099581113BC1D801ED91FC9180
:102730000284F385E02D68E070E0C80109958111FD
:102740002FC1D801ED91FC910284F385E02D69E061
:1027500070E0C8010995811123C1D801ED91FC9168
:102760000284F385E02D6AE070E0C80109958111CB
:1027700017C1D801ED91FC910284F385E02D6CE046
:1027800070E0C801099581110BC1D801ED91FC9150
:102790000284F385E02D64E070E0C80109958111A1
:1027A000FFC01E82FDC063E070E0C8010995882368
:1027B00051F08F8198858230910514F0019719C0EE
:1027C00081E090E016C0D801ED91FC910284F38580
:1027D000E02D62E070E0C8010995882369F02F813F
:1027E000388589859A8501972817390714F4C90116
:1027F000019698878F83B6C0D801ED91FC91028431
:10280000F385E02D61E070E0C8010995882361F04F
:1028100029853A858F8198850196821793070CF058
:1028200051C0C90101974EC0D801ED91FC910284BD
:10283000F385E02D60E070E0C8010995882351F030
:1028400089859A858E37910514F401963BC08EE7F1
:1028500090E038C0D801ED91FC910284F385E02D21
:1028600064E070E0C80109958823D1F08B81813044
:1028700049F0823071F087E190E098878F8385E29C
:1028800090E020C084E190E098878F8380E290E020
:1028900019C08EE190E098878F8389E290E012C0A2
:1028A000D801ED91FC910284F385E02D6CE070E09D
:1028B000C8010995882349F088E090E098878F83C4
:1028C0008AE290E09A8789874DC0D801ED91FC910A
:1028D0000284F385E02D68E070E0C8010995882343
:1028E00069F082E08B838EE190E09E878D8789E29C
:1028F00090E09C878B8789E490E032C0D801ED910D
:10290000FC910284F385E02D6AE070E0C80109952E
:10291000882379F081E08B8324E130E03E872D87A6
:1029200020E230E03C872B8725E330E0388B2F878F
:102930001AC0D801ED91FC910284F385E02D69E085
:1029400070E0C8010995882359F11B8287E190E066
:102950009E878D8785E290E09C878B8787E490E057
:10296000988B8F8781E08E831BC08091E1029091CC
:10297000E202009799F06F810E9481068091E10246
:102980009091E202698501960E9481068091E102A0
:102990009091E2026B8102960E9481061D821C8248
:1029A000DF91CF911F910F91FF90EF90DF900895ED
:1029B0000F931F93CF93DF93EC011A8289E391E089
:1029C000998388831B820091E1021091E202011534
:1029D0001105F1F581E00E94640D8C019093E202F3
:1029E0008093E102892BA1F563E070E081E00E9411
:1029F000D90C9093E2028093E1021B8227E130E040
:102A00003E872D8725E230E03C872B8727E430E0A6
:102A1000388B2F8728E030E038872F832AE230E098
:102A20003A872987009731F168E00E9481068091FA
:102A3000E1029091E202698501960E9481068091EF
:102A4000E1029091E2026B8102960E94810612C01F
:102A5000C8010E94511B90E098878F83C80101969E
:102A60000E94511B90E09A878987C80102960E94B4
:102A7000511B8B838B81813069F08230B1F087E10B
:102A800090E09E878D8785E290E09C878B8787E426
:102A900090E015C084E190E09E878D8780E290E011
:102AA0009C878B8785E390E00AC08EE190E09E874B
:102AB0008D8789E290E09C878B8789E490E0988BF2
:102AC0008F8789859A858038910524F08EE790E07C
:102AD0009A87898789859A852F81388582179307F8
:102AE0001CF4019798878F8381E090E09D838C830D
:102AF000DF91CF911F910F9108958091E302909102
:102B0000E402892BF9F480E00E94640D9093E402C2
:102B10008093E302892BB1F462E070E080E00E94D0
:102B2000D90C9093E4028093E302009759F061E09E
:102B30000E9481068091E3029091E40260E0019698
:102B40000C94810608950F931F93CF93DF938C010C
:102B5000EB01FC018381E881F981882359F0068427
:102B6000F785E02DCB010995882309F4EAC0F80127
:102B70001382E7C00284F385E02D64E070E0CE01AB
:102B80000995882381F083E090E00E94D31DFC0129
:102B900012822CE232E031832083BC01CE010E94FC
:102BA0009A0D80E017C0E881F9810284F385E02D59
:102BB00061E070E0CE010995882391F081E190E019
:102BC0000E94D31D8C010E94D814B801CE010E942E
:102BD0009A0D81E0DF91CF911F910F910C94A91272
:102BE000E881F9810284F385E02D6EE070E0CE018A
:102BF00009958823D1F082E090E00E94D31D8C01DA
:102C000084E192E0F801918380838C819D8100971B
:102C100011F00E946B1E1D830C838E819F819B830C
:102C20008A831F821E8280E086C0E881F981028447
:102C3000F385E02D63E070E0CE010995882369F00B
:102C400088E190E00E94D31D8C010E94200CB80105
:102C5000CE010E949A0D82E0BDCFE881F981028405
:102C6000F385E02D69E070E0CE0109958823D1F06D
:102C700082E090E00E94D31D8C0186E292E0F80190
:102C8000918380838C819D81009711F00E946B1E3F
:102C90001D830C838E819F819B838A831F821E826A
:102CA00081E049C0E881F9810284F385E02D6AE082
:102CB00070E0CE0109958823D1F082E090E00E9477
:102CC000D31D8C0180E292E0F801918380838C8196
:102CD0009D81009711F00E946B1E1D830C838E81D5
:102CE0009F819B838A831F821E8282E024C0E881A9
:102CF000F9810284F385E02D6BE070E0CE01099547
:102D00008823F9F082E090E00E94D31D8C018AE1D3
:102D100092E0F801918380838C819D81009711F06E
:102D20000E946B1E1D830C838E819F819B838A83EF
:102D30001F821E8283E0DF91CF911F910F910C942F
:102D40009C12DF91CF911F910F910895CF92DF9246
:102D5000EF92FF920F931F93CF93DF936C017A0151
:102D60008B01C0E0D0E0CE15DF0581F0D8016D9178
:102D70008D01D601ED91FC910190F081E02DC6010D
:102D80000995892B11F02196EECF7E01C701DF91C5
:102D9000CF911F910F91FF90EF90DF90CF9008950A
:102DA000089580E090E00895FC01538D448D252F17
:102DB00030E0842F90E0821B930B541710F0CF96D5
:102DC000089501970895FC01918D828D981761F007
:102DD000828DDF01A80FB11D5D968C91928D9F5F52
:102DE0009F73928F90E008958FEF9FEF0895FC01FD
:102DF000918D828D981731F0828DE80FF11D858DB0
:102E000090E008958FEF9FEF08950E94F41E82E4F2
:102E100092E00E94930621E0892B09F420E0822FA2
:102E20000895EF92FF920F931F93CF93DF93EC01DE
:102E300081E0888F9B8D8C8D981305C0E889F98976
:102E4000808185FD26C0F62E0B8D10E00F5F1F4F91
:102E50000F731127E02E8C8DE8120CC00FB607FC03
:102E6000FACFE889F989808185FFF5CFCE010E94EC
:102E7000FE0BF1CF8B8DFE01E80FF11DE35AFF4FE2
:102E8000F0829FB7F8940B8FEA89FB89808180627A
:102E90000AC09FB7F894EE89FF896083E889F989B1
:102EA00080818370806480839FBF81E090E0DF91A8
:102EB000CF911F910F91FF90EF900895CF93DF93E3
:102EC000EC01888D8823C9F0EA89FB89808185FD22
:102ED00005C0A889B9898C9186FD0FC00FB607FC83
:102EE000F5CF808185FFF2CFA889B9898C9185FFC4
:102EF000EDCFCE010E94FE0BE7CFDF91CF91089579
:102F00001F920F920FB60F9211242F933F938F931E
:102F10009F93AF93BF938091EB029091EC02A091AD
:102F2000ED02B091EE023091EA0223E0230F2D373B
:102F300020F40196A11DB11D05C026E8230F0296BD
:102F4000A11DB11D2093EA028093EB029093EC0245
:102F5000A093ED02B093EE0280913B0290913C026F
:102F6000A0913D02B0913E020196A11DB11D80933A
:102F70003B0290933C02A0933D02B0933E02BF916E
:102F8000AF919F918F913F912F910F900FBE0F9016
:102F90001F9018951F920F920FB60F9211242F9326
:102FA0003F934F935F936F937F938F939F93AF93D1
:102FB000BF93EF93FF9382E492E00E94FE0BFF9198
:102FC000EF91BF91AF919F918F917F916F915F91A1
:102FD0004F913F912F910F900FBE0F901F9018951A
:102FE0001F920F920FB60F9211242F938F939F93DE
:102FF000EF93FF93E0915202F09153028081E091B0
:103000005802F091590282FD12C0908180915B02BA
:103010008F5F8F7320915C02821751F0E0915B0209
:10302000F0E0EE5BFD4F958F80935B0201C08081E5
:10303000FF91EF919F918F912F910F900FBE0F9065
:103040001F901895E2E4F2E01382128288EE93E07A
:10305000A0E0B0E084839583A683B78387E291E004
:103060009183808385EC90E09587848784EC90E061
:103070009787868780EC90E0918B808B81EC90E045
:10308000938B828B82EC90E0958B848B86EC90E026
:10309000978B868B118E128E138E148E1092E002F7
:1030A0001092DF021092E2021092E1021092E4020A
:1030B0001092E3020895CF93DF9300D01F92CDB713
:1030C000DEB7789484B5826084BD84B5816084BDA8
:1030D00085B5826085BD85B5816085BD80916E00B6
:1030E000816080936E0010928100809181008260E7
:1030F0008093810080918100816080938100809124
:1031000080008160809380008091B1008460809312
:10311000B1008091B00081608093B00080917A000E
:10312000846080937A0080917A00826080937A0034
:1031300080917A00816080937A0080917A00806823
:1031400080937A001092C100E0915202F0915302F4
:1031500082E08083E0914E02F0914F021082E09174
:103160005002F091510280E1808310925A02E09166
:103170005602F091570286E08083E0915402F0916C
:103180005502808180618083E0915402F091550264
:10319000808188608083E0915402F09155028081A3
:1031A00080688083E0915402F091550280818F7D88
:1031B000808380910A0190910B01019790930B01FC
:1031C00080930A0143E050E062E070E0CE01019696
:1031D0000E94411B8981853A31F48A818E3919F424
:1031E0008B818C3811F080E04DC089E090E00E9426
:1031F000511B8233A1F162E389E090E00E948106D5
:10320000109241021092400260E080E090E00E9443
:1032100081066091400281E090E00E9481068091E9
:10322000BB019091BC01A091BD0189839A83AB83BE
:10323000CE0101967C0102E010E0D701DD907D0116
:10324000C8010E94511BD81621F06D2DC8010E94A3
:10325000591B0F5F1F4F0530110579F712C080E031
:1032600090E00E94511B90E09093410280934002B5
:1032700081E090E00E94511B90E090934102809386
:10328000400281E08093E90288E491E00E94D31D2E
:10329000FC0122EC31E02193319321E2DF011D9208
:1032A0002A95E9F7FC0113A69093E8028093E702C0
:1032B0008CEB90E00E94D31D2EEF31E0DC011196E3
:1032C0003C932E939C012E583F4F1D963C932E937A
:1032D0001C9720E430E01B963C932E931A971E9681
:1032E0001C921E9791961C9291972AE0E0EFF1E0D4
:1032F000579601900D922A95E1F79093E6028093FC
:10330000E50283E00E942B1283E00E9403120E94D8
:103310007D158091E3029091E402009749F00196B7
:103320000E94511B823091F08330D1F0813039F00E
:1033300082E090E00E94D31D24E132E00DC082E0E3
:1033400090E00E94D31D26E232E010C082E090E0BF
:103350000E94D31D20E232E0FC013183208309C0AA
:1033600082E090E00E94D31D2AE132E0DC012D933F
:103370003C936C010E947D158091E3029091E402E0
:10338000009731F00E94511B813071F08230A1F022
:1033900083E090E00E94D31DFC0112822CE232E017
:1033A000318320838C010FC081E190E00E94D31D06
:1033B0008C010E94D81407C088E190E00E94D31DC0
:1033C0008C010E94200CA090E702B090E802E090EF
:1033D000E502F090E60285E00E942B1285E00E9453
:1033E000031284E00E942B1284E00E940312D70192
:1033F0001996BC92AE92189712960C931297139648
:103400001C9313971496CC9214971596DC921597EB
:1034100017961C921E92169732E3632E32E0732E9B
:103420005524539448E0242E312C8091E9028823BE
:1034300009F41CC18091E7029091E802DC01ED9152
:10344000FC910190F081E02D09958111F7C0009168
:10345000E5021091E602F8018685C484D584A28431
:10346000B384882351F1E12CF12CEA14FB0464F5B8
:10347000C701F7FC079623E0959587952A95E1F714
:10348000F601E80FF91F2081022E000C330BC70153
:10349000B1010E94A51D02C0359527958A95E2F7D6
:1034A000C9018170992720FF02C081E390E00E944A
:1034B0007212FFEFEF1AFF0AD8CF7601C7018C19FD
:1034C0009D098A159B057CF08AE090E00E947212AB
:1034D000D801ED91FC910484F585E02DC801099592
:1034E00081110EC038C0F70181917F01882319F046
:1034F00081E390E002C080E090E00E947212DECF93
:10350000D8011296ED91FC911397309719F08281B2
:10351000811121C084E090E00E94D31D7C01FC0158
:103520007182608253825282892B09F4A2C0F80111
:1035300086819781009711F00E946B1ED801129628
:103540008D919C91139717969C938E931697139633
:10355000FC92EE921297C0900A01D0900B010D2CB4
:10356000000CEE08FF080E9477124B015C01C114A9
:10357000D104E104F104F1F00E947712DC01CB01E7
:1035800088199909AA09BB09883E9340A105B1058C
:1035900070F3F1E0CF1AD108E108F10828EE820EAD
:1035A00023E0921EA11CB11CC114D104E104F1045A
:1035B00019F7DDCFF8940091E5021091E602D801E9
:1035C000ED91FC910480F581E02DC8010995F80189
:1035D00080859185DC01ED91FC910084F185E02DE1
:1035E0000995F80182819381009751F040855185BA
:1035F000DC01ED91FC910190F081E02DB80109957D
:10360000F80186819781892B71F4848195810097D7
:1036100051F040855185DC01ED91FC910190F081E4
:10362000E02DB80109958091E7029091E802DC0154
:10363000ED91FC910480F581E02D09958091E702E0
:103640009091E802DC01ED91FC910280F381E02D84
:103650000995F8948091E7029091E802DC01ED91E0
:10366000FC910680F781E02D099578940E949F06D1
:10367000DCCEF8018681978193838283178216823C
:103680006ACFDC01CB01FC01F999FECF06C0F2BD87
:10369000E1BDF89A319600B40D9241505040B8F710
:1036A0000895F999FECF92BD81BDF89A992780B50A
:1036B0000895262FF999FECF1FBA92BD81BD20BD76
:1036C0000FB6F894FA9AF99A0FBE019608955058D9
:1036D000BB27AA270E947F1B0C94F91C0E94EB1C9D
:1036E00038F00E94F21C20F039F49F3F19F426F4C0
:1036F0000C94E81C0EF4E095E7FB0C94E21CE92F17
:103700000E940A1D58F3BA176207730784079507CA
:1037100020F079F4A6F50C942C1D0EF4E0950B2EF8
:10372000BA2FA02D0B01B90190010C01CA01A00113
:103730001124FF27591B99F0593F50F4503E68F16E
:103740001A16F040A22F232F342F4427585FF3CFAF
:10375000469537952795A795F0405395C9F77EF480
:103760001F16BA0B620B730B840BBAF09150A1F0C9
:10377000FF0FBB1F661F771F881FC2F70EC0BA0F4F
:10378000621F731F841F48F4879577956795B795D7
:10379000F7959E3F08F0B0CF9395880F08F09927D2
:1037A000EE0F9795879508950E94BE1C08F481E05E
:1037B00008950E94ED1B0C94F91C0E94F21C58F015
:1037C0000E94EB1C40F029F45F3F29F00C94E21CAE
:1037D00051110C942D1D0C94E81C0E940A1D68F3D5
:1037E0009923B1F3552391F3951B550BBB27AA27BA
:1037F00062177307840738F09F5F5F4F220F331FF4
:10380000441FAA1FA9F335D00E2E3AF0E0E832D0BB
:1038100091505040E695001CCAF72BD0FE2F29D0BE
:10382000660F771F881FBB1F261737074807AB0790
:10383000B0E809F0BB0B802DBF01FF2793585F4F05
:103840003AF09E3F510578F00C94E21C0C942D1D2B
:103850005F3FE4F3983ED4F3869577956795B795E7
:10386000F7959F5FC9F7880F911D9695879597F9F2
:103870000895E1E0660F771F881FBB1F621773076B
:103880008407BA0720F0621B730B840BBA0BEE1F80
:1038900088F7E09508950E94521C6894B1110C9429
:1038A0002D1D08950E94121D88F09F5798F0B92F82
:1038B0009927B751B0F0E1F0660F771F881F991F65
:1038C0001AF0BA95C9F714C0B13091F00E942C1DBE
:1038D000B1E008950C942C1D672F782F8827B85FCE
:1038E00039F0B93FCCF3869577956795B395D9F7BD
:1038F0003EF490958095709561957F4F8F4F9F4FC7
:103900000895E89409C097FB3EF4909580957095D2
:1039100061957F4F8F4F9F4F9923A9F0F92F96E91B
:10392000BB279395F695879577956795B795F11190
:10393000F8CFFAF4BB0F11F460FF1BC06F5F7F4F2D
:103940008F4F9F4F16C0882311F096E911C077233F
:1039500021F09EE8872F762F05C0662371F096E848
:10396000862F70E060E02AF09A95660F771F881F17
:10397000DAF7880F9695879597F90895990F0008BB
:10398000550FAA0BE0E8FEEF16161706E807F90731
:10399000C0F012161306E407F50798F0621B730BCC
:1039A000840B950B39F40A2661F0232B242B252B4D
:1039B00021F408950A2609F4A140A6958FEF811DF0
:1039C000811D089597F99F6780E870E060E0089591
:1039D0009FEF80EC089500240A9416161706180627
:1039E0000906089500240A94121613061406050603
:1039F0000895092E0394000C11F4882352F0BB0F94
:103A000040F4BF2B11F460FF04C06F5F7F4F8F4FF6
:103A10009F4F089557FD9058440F551F59F05F3F31
:103A200071F04795880F97FB991F61F09F3F79F0E0
:103A300087950895121613061406551FF2CF469562
:103A4000F1DF08C0161617061806991FF1CF8695E4
:103A50007105610508940895E894BB2766277727C8
:103A6000CB0197F908950E94BE1C08F48FEF0895CA
:103A70000E944B1D0C94F91C0E94EB1C38F00E9414
:103A8000F21C20F0952311F00C94E21C0C94E81C1D
:103A900011240C942D1D0E940A1D70F3959FC1F3F3
:103AA000950F50E0551F629FF001729FBB27F00DEC
:103AB000B11D639FAA27F00DB11DAA1F649F662741
:103AC000B00DA11D661F829F2227B00DA11D621F90
:103AD000739FB00DA11D621F839FA00D611D221F4A
:103AE000749F3327A00D611D231F849F600D211D2E
:103AF000822F762F6A2F11249F5750409AF0F1F0B1
:103B000088234AF0EE0FFF1FBB1F661F771F881F19
:103B100091505040A9F79E3F510580F00C94E21C53
:103B20000C942D1D5F3FE4F3983ED4F38695779572
:103B30006795B795F795E7959F5FC1F7FE2B880FBF
:103B4000911D9695879597F9089597FB072E16F482
:103B5000009407D077FD09D00E94B91D07FC05D05D
:103B60003EF4909581959F4F0895709561957F4F94
:103B70000895AA1BBB1B51E107C0AA1FBB1FA617B4
:103B8000B70710F0A61BB70B881F991F5A95A9F706
:103B900080959095BC01CD010895EE0FFF1F059013
:103BA000F491E02D09940F931F93CF93DF9382300C
:103BB000910510F482E090E0E091F102F091F202C0
:103BC00020E030E0A0E0B0E0309719F14081518171
:103BD0000281138148175907C8F08417950769F4C3
:103BE000109731F012960C93129713961C9327C0DE
:103BF0000093F1021093F20222C02115310519F051
:103C00004217530718F49A01BD01EF01DF01F801D3
:103C1000DBCF21153105F9F0281B390B2430310594
:103C200080F48A819B816115710521F0FB019383EA
:103C3000828304C09093F2028093F102FE013296D7
:103C400044C0FE01E20FF31F81939193225031098A
:103C5000398328833AC02091EF023091F002232B60
:103C600041F420910E0130910F013093F002209326
:103C7000EF0220910C0130910D012115310541F425
:103C80002DB73EB74091100150911101241B350B07
:103C9000E091EF02F091F002E217F307A0F42E1B7F
:103CA0003F0B2817390778F0AC014E5F5F4F2417A0
:103CB000350748F04E0F5F1F5093F0024093EF021C
:103CC0008193919302C0E0E0F0E0CF01DF91CF91CA
:103CD0001F910F910895CF93DF93009709F481C04E
:103CE000FC01329713821282A091F102B091F2028C
:103CF000109781F420813181820F931F2091EF0270
:103D00003091F0022817390751F5F093F002E09353
:103D1000EF0267C0ED0120E030E0CE17DF0740F48E
:103D20004A815B819E0141155105F1F0EA01F5CF11
:103D3000D383C28340815181840F951FC817D9074F
:103D400059F488819981840F951F0296918380830D
:103D50008A819B81938382832115310529F4F09315
:103D6000F202E093F1023DC0E901FB83EA8349914D
:103D70005991C40FD51FEC17FD0761F48081918123
:103D8000840F951F0296E90199838883828193812C
:103D90009B838A83E0E0F0E012968D919C911397CB
:103DA000009719F0FD01DC01F7CF8D919C911197DF
:103DB0009D012E5F3F4F820F931F2091EF023091A4
:103DC000F0022817390769F4309729F41092F202AB
:103DD0001092F10202C013821282B093F002A093FB
:103DE000EF02DF91CF91089581E090E0F8940C9478
:103DF000001FDC0101C06D9341505040E0F7089571
:043E0000F894FFCF64
:103E0400090003000000000001010C000000F3029F
:103E1400800000807F7F7F7F00004003000000005F
:103E2400007C07000000001117A616D4165E179335
:103E340006E316F71600000000B312001011121367
:103E4400141516171718191A1B1B1C1D1E1E1F20CC
:103E5400212222232424252626272828292A2A2BFE
:103E64002C2C2D2D2E2F2F3030313132333334344E
:103E740035353636373738383839393A3A3B3B3BBB
:103E84003C3C3D3D3D3E3E3F3F3F40404040414144
:103E940041424242434343434344444444444545EA
:103EA40045454546464646464646464646474747AE
:103EB4004747474747474747474747A59E8C000022
:103EC4000000F806F506FA0B810B710767075F0718
:103ED400510745070107FB06060700000000000024
:103EE400000005170517051705170517051705170A
:103EF4000080808080800000020200000000D80C56
:103F04007F0BBE09ED06E506C806BC06B206A90687
:103F140000000000230300000000870000000000F0
:103F2400D50100000000A704000000007104000097
:0A3F34000000A315000000000517AF
:00000001FF
